:020000020000FC
:10000000E1CD00000000000020C0AEC18EC00000A5
:10001000000098C000000000000000000203040679
:10002000080C10182030406080000406080C1018DE
:100030002030406080A0C0000003070F1F000D0D9E
:1000400004050D050305030302004FB662FD0CC055
:10005000552041F00994C52DC095089483FDC7959E
:10006000C4BD64604FBE1895C0916400089483FDC0
:10007000C795C4BD6B7FC0916400CF3F09F41EC01B
:1000800070FF1AC082FD05C04FBE93989498959852
:10009000189576FD0EC064FD0CC0C091B100C0FD86
:1000A0009298C1FDC298C2FDC198CAEFC095CA9589
:1000B000F1F79398949895984FBE189524BCCC2747
:1000C000C064C8BF6460F8CFC6CF70FFC4CF64FD02
:1000D000C2CF939AC0CF70FFBECF64FDBCCF949ABD
:1000E000BACF70FFB8CF64FDB6CF959AB4CF929ACD
:1000F00070FFB1CF64FDAFCFC7E0CA95F1F7939A17
:10010000AACFC29A70FFA7CF64FDA5CFC7E0CA955A
:10011000F1F7949AA0CFC19A70FF9DCF64FD9BCF59
:10012000C7E0CA95F1F7959A96CF4FB6C9B7CF7E7B
:10013000C9BF6E7FCCB5CE0DDDB5DF1DDBBDCABD41
:100140004FBE18953FB68F7EA9B7A072A2118061ED
:10015000A9B7AF7DA9BFA9B7AE7FA9BF7894A09179
:100160006800AA2341F085FD2FC0A0916800AA95E0
:10017000A093680029C040E050E085FD15C0A6B3FB
:1001800096FDA095A0FD4FEFAEB5A06496FDAF7BA8
:10019000AEBDAA27A062A8BF8D7FA6B396FDA0958D
:1001A000A0FD5FEF451739F7A8E161FDA093680056
:1001B00085FD03C0A8E1A09368004093960081608C
:1001C000442311F02092990085FD0EC0A091690092
:1001D000AA2331F0A0916900AA95A093690004C0F8
:1001E0008061AA27A062A8BF80FF3CC0A0919600B2
:1001F0004A2F61FF8E7F85FD1CC0A091B400A43002
:10020000C1F4403F08F040EFA42FA295AF704A0F11
:100210005091B600533069F0A695A69550FD01C0E7
:10022000A69552FD03C0A41B4A2F03C04A0F08F431
:100230004FEF40936100A72FA670A1F073FD12C08D
:10024000A0917000AA0FAA0F50919E005695569546
:10025000541708F0452F4A0F4093610018F4AFEF90
:10026000A09361004091B400443009F03EC0A091D9
:100270006100A093630040916300A0919B004A1726
:1002800008F04A2FA0919D004A1708F04A2F542EDB
:10029000A091A000AA2309F422C0542F5A1B10F4E5
:1002A000A42F50E0BA2E8894AA1FAA2EA091A200D3
:1002B000A095AA22A50E58F0A091A100A21509F0C0
:1002C000AA95AA0EA093A10048F04A2D08C0A091BB
:1002D000A100BA1608F0A395A093A1004FEF409398
:1002E00064007F7B485F08F07064A0916000A39574
:1002F000A093600059F0F894A9B7A160A9BF84FF4A
:1003000003C0A9B7A062A9BF3FBE1895A091740011
:10031000A395A093740041E050916800552329F003
:1003200085FF03C05A9550936800A0919600A130B4
:1003300018F0209299000DC020929A002092A300FC
:10034000A0919900AF5FA093990018F0AFEFA09330
:100350009900F894A9B7A160A9BF84FF03C0A9B709
:10036000A062A9BF3FBE18953FB646B557B58F7E70
:10037000A9B7A072A2118061A9B7AF7DA9BFA9B723
:10038000AE7FA9BF789481FD25C0AEB5AF7B96FD49
:10039000A064AEBD8260A6B396FDA095A0FF05C087
:1003A000409365005093660041C1AEB5A06496FDD0
:1003B000AF7BAEBDAA27A062A8BF8D7F85FF01C01D
:1003C00028C140E0A6B396FDA095A0FD22C14093B0
:1003D000960011C1AEB5A06496FDAF7BAEBD8D7F1A
:1003E00061FF72C0AEB5AF7B96FDA064AEBDAA271B
:1003F000A062A8BF82604093910050939200A090A9
:100400008F004A19B09090005B09BB24A22C4C3895
:10041000520518F42092950049C0A091D400AA2357
:1004200059F1483C520528F4A0E1BA2EAAE0AA2EC0
:1004300023C04836A1E05A0728F4A8E0BA2EAFE05E
:10044000AA2E1AC0403DA2E05A0728F4A4E0BA2E12
:10045000AEE1AA2E11C0403AA5E05A0728F4A2E066
:10046000BA2EACE3AA2E08C04839A8E05A0720F4F7
:10047000A1E0BA2EA8E7AA2EC42EA0919300CA1A12
:10048000D52EA0919400DA0ADD202AF4AFEFC094B3
:10049000D094CA1ADA0A20929500A8E0A210A0E02F
:1004A000CA14DA0618F4A1E0A093950040939300D3
:1004B00050939400409191005091920040938F008E
:1004C0005093900042E097C0A09165004A1BA09114
:1004D00066005A0B94FD82C093FD80C092FD7CC0E3
:1004E00086FF03C0D52EC42E0CC05695479591FDAE
:1004F00073C05695479590FD6FC0D52EC42ED694E7
:10050000C79461FD19C0AC2DAC51AD2DA24008F0CF
:1005100005C0DD2089F4AC2DA85C70F4A0916700C3
:10052000A395AA2311F0A0936700AA3008F471C024
:100530002092960081606DC0A0916700AA2319F0F7
:10054000AA95A0936700A22C5091BA0097FD06C00F
:10055000A090C800533011F4A090D000AAEFAA0ECA
:10056000A22DA21DCA18DA0A4FB74170533049F4C0
:10057000442321F087FD05C0806803C087FF01C0C8
:100580008F77442359F0533031F4AFEFC094D094B7
:10059000CA1ADA0A03C040E050E020C0533049F4E0
:1005A000CC0CDD1CAAE0CA1AD20818F4A0E0CA2EAE
:1005B000D22CAFEFCA16D20418F04FEF50E00EC0A5
:1005C000A091AC00CA9E412D000C441F50E008F0E1
:1005D00012C04FEF50E00FC05695479594FF07C0EB
:1005E000552309F04FEFA42FA6954A0F521D4F3FF8
:1005F000520508F04FEF40939600816061FF09C0FB
:10060000AFE1A095A923AB299A2F8F7DBB2009F4D8
:100610008062A8E1A093680085FF03C0AAE0A093D0
:10062000680061FD03C085FD01C08F7E85FD03C0AC
:10063000A6E0A0936900F894A9B7A160A9BF84FFC0
:1006400003C0A9B7A062A9BF3FBE189511E00AC0B8
:1006500013E008C01AE006C01EE104C014E602C0A0
:1006600018EC00C005E1BB27BA95F1F70A95D9F758
:100670001A95C1F708952AE338E709C020E33CE85A
:1006800006C02AE234EB03C025E238EC00C0B0918A
:10069000AD00BA9509F4089512E0BB27C29ABA9545
:1006A000F1F7949ABA95F1F79498BA95F1F7C29840
:1006B000BA95F1F7123009F0939A123009F4959A2D
:1006C000B091AD00BA95F1F7123009F0939812305D
:1006D00009F49598B7E8BA95F1F71A95F1F6022F53
:1006E000B22FBA95F1F70A95D9F73A9581F6C29AE1
:1006F0000895221B39E0001F3A9509F40895221F3E
:10070000211B18F4210F8894F6CF0894F4CF622CA3
:10071000722CB0E08894B395221F331FE0F7379511
:1007200027958894912E802E020B130B10F4192D0F
:10073000082D10F4889401C00894661C771CBA95A3
:1007400071F7172D062D0895322D11232AF43A95AD
:1007500000951095031B130BF894029F712C002D2C
:10076000129F912C802C7894780C172D921C292D97
:10077000B4E06B2E2695179507956A94D9F7332325
:1007800021F000951095031B130B08950091B40000
:100790000430A1F1B0919600B15008F010C0B091B2
:1007A0006100B093630020927E0020927F0020922F
:1007B000800020928100209282006F7D1FC0609097
:1007C000B4006062B0916100B093620008E317EC7E
:1007D00020917A0030917B0036952795B62DBA95F9
:1007E00041F036952795B62DBA95BA9511F0369504
:1007F00027958DDF00937E0010937F000895009170
:100800007E00B09162000B1B10917F00120928F44A
:100810000038BFEF1B0740F009C00F37120508F47E
:1008200005C00FE710E002C000E81FEF009383004F
:1008300010938400089500918300B09180000B0F05
:1008400010918400B09181001B1F20E03091840042
:1008500033230AF42A95B09182002B1F1AF4203F0B
:1008600040F00AC02F3008F407C00FEF1FEF2FE051
:1008700003C000E010E020EF30916300B0919B00D6
:100880003B1718F4323030F009C0B0918400BB231C
:100890005AF004C0B0918400BB2332F4009380006E
:1008A000109381002093820008952091D700009139
:1008B0008300000F10918400111F46DF11232AF4DA
:1008C0000038BFEF1B0740F009C00F37120508F4CE
:1008D00005C00FE710E002C000E81FEF002352F050
:1008E000B0916200B01B0B2F18F0013008F00AC065
:1008F00001E008C000950F5FB09162000B0F08F097
:1009000001C00FEF0093850008952091D800009159
:1009100081001091820018DF11232AF40130BFEF0B
:100920001B0740F009C00F3F120508F405C00FEF88
:1009300010E002C001E01FEF112352F0B0918500DA
:10094000B01B0B2F18F0013008F00AC001E008C0FE
:1009500000950F5FB09185000B0F08F001C00FEFFD
:100960000093630008950FEF71FD1EC0B091D30096
:10097000BB23D1F0B0917B00BB23B1F00FEF1091FE
:100980007B00B7DEF894B091730072FDB5E00B9F69
:10099000112D002D7894112309F00FEFB0919E00D6
:1009A0000B1710F400919E0000939D000895009194
:1009B0007A0010917B0000541140B0919D0010F41A
:1009C000BA9501C0B39511F0B0939D00089500C091
:1009D00008952091B500B6B1B6FDFBCF04B115B1B5
:1009E000B6B1BF77B6B9B091AA00B395B093AA00DB
:1009F000B83060F12092AA00B091D200BB2321F15F
:100A0000112329F0B091AB00BF3F61F009C0B09154
:100A1000AB000B1739F020F4BB2321F0BA9502C0CC
:100A2000B395E1F300919B00B093AB00B93B50F458
:100A300000ECBA3A38F400E8BB3920F400E4BC38E2
:100A400008F400E000939B007F7E089510919B00C6
:100A5000B0E11B0F08F41FEF10939B00B091B4009E
:100A6000B43081F000919B00B0916300B01B10F492
:100A700000916300B0919D000B1708F00B2F502ED2
:100A800000936400B091AA00B73009F47061089532
:100A900002E3F894B091D9000B9F012D000C001FC8
:100AA0007894B0919B000B1710F000919B0000937D
:100AB000610000936300502E0093640000939E0039
:100AC000089520927A00B0EFB0937B000895F894D7
:100AD0000CB51DB52091740078943091750060902C
:100AE00076000093750010937600031B160971FDC4
:100AF00003C077FD80C028C07090770020937700F6
:100B00002709222319F00FEF1FEF0EC08090780005
:100B10009090790030937800609279000091750090
:100B2000109176000819190920917A0030917B0004
:100B300036952795020F131F10F40FEF1FEF009348
:100B40007A0010937B002BC020917A0030917B00BB
:100B50003901B4E08B2EB2E09B2E343040F08A9401
:100B60009A94383020F072FD02C08A949A94769458
:100B700067948A94E1F726193709992021F0169590
:100B800007959A94E1F7200F311F20937A00309354
:100B90007B0028F43FEF30937A0030937B003230B3
:100BA00008F4706871FF02C0B3E00DC0B091C400DA
:100BB00000917100023838F0B395003A08F0B3950F
:100BC000B63008F0B5E09B2EB4E08B2E10917B0080
:100BD00000917A0024E0169507952A95E1F7081907
:100BE000120928F0B02FB250B12FB20910F402E070
:100BF00010E0980126C020917A0030917B003901E5
:100C000076946794669466946694261932090695DC
:100C10000695200F321D20937A0030937B003230EE
:100C200008F07F7704E03695279536952795269529
:100C30002695201B10F0223008F422E089019090C4
:100C4000C40060FDFECFE0908B00F0908C006160EE
:100C5000B9B7B061B9BF380177FD41C076946794E8
:100C600000938B0010938C00B92DB330E1F0B0FDF0
:100C700004C0060D171D930106C0000F111F02507E
:100C8000120922E030E0B92DB33068F020938D00D6
:100C900030938E0000938700109388006092890043
:100CA00070928A003AC000938D0010938E002093BA
:100CB0008700309388006092890070928A0071FFEB
:100CC0000DC0BFE0B0938D0020928E00B0938900DC
:100CD00020928A00B0938B0020928C001EC06694F4
:100CE00000938B00B92DB33091F0B0FD03C0060D19
:100CF000262D03C0000F025022E0B92DB33038F08A
:100D000020938D00009387006092890006C00093B5
:100D10008D00209387006092890000917C0002FD85
:100D20000350013049F495FD12C0B0B7B860B0BFB0
:100D3000B0E0B06CB7B90EC0023039F4B0B7B860EB
:100D4000B0BFB1E0B06CB7B905C095FDEECFB0B79C
:100D5000B77FB0BF0091A200000F10F4BBE60B27D5
:100D60000093A20060FDFECFB2E0B0936E00616020
:100D7000B9B7B061B9BFB72FB670D1F020917A0082
:100D800030917B00369527953695279571FF02C0E7
:100D9000B0E43B0FF8940CB51DB5020F131F1BBD3B
:100DA0000ABD6160B0E1B8BFB9B7B061B9BF7894AE
:100DB0000895686020927D0020E066FD20E206C074
:100DC000686020927D0020E266FD20E001E011E0F5
:100DD00077FD11C0B72FB67009F0677F14E100915D
:100DE0007B00069509F403950F3008F00FE071FFC2
:100DF00002C004E114E160FD0FC0B0917D00BB238F
:100E000059F071FF06C0B0916E00BA95B0936E00B4
:100E100011F4706251C0ABDFB0B73B2FB77FB0BFEA
:100E2000B8B1B0B733FDB860B0BFB0917D00B39535
:100E3000B0937D00B8B177FD06C0B1E071FDB3E0BD
:100E4000BA95F1F7B8B1B072B21709F02AC071FFC4
:100E500005C00395011708F00A95CDCF63FD05C0C5
:100E60000395011708F0B2CFC6CF677FF8943CB561
:100E70006DB470907A00B0917B00770CBB1F08F4C2
:100E8000BFEF770CBB1F08F4BFEF370D6B1E6BBCB9
:100E90003ABD6160B0E1B8BFB9B7B061B9BF78948D
:100EA00095CFB0916D00B13008F490CF63FD8ECF37
:100EB0000A9509F0A0CF7F7D20918D0030918E00A2
:100EC000F894B0E1B8BF0CB51DB5020F131F1BBDE0
:100ED0000ABDE0908700F09088006160B9B7B0610A
:100EE000B9BF7894B72FB67039F0B0916D0072FF2A
:100EF000B395B0936D0009C075FF07C066FD05C0CE
:100F000063FD03C0BF91BF9109C5089500E063FF71
:100F100001C001E0F89410917100B7E01B9F212DF2
:100F2000102D7894200F26951795269517952695C0
:100F3000179510937100183718F4B8E7B093710043
:100F400000917100B09172000B1720F060619398CE
:100F50009498959860FDFECFE0908900F0908A000B
:100F60006160B9B7B061B9BF0895AC98B2E095FDC2
:100F70000AC0F894B0937C00C29A929862FF01C0B4
:100F8000959A7894F9C0F894B0937C00C29AC1986D
:100F900062FF01C0939A7894EFC0AC9AB3E082FFED
:100FA00024C095FD11C002E0F894B0937C00E1E804
:100FB000F0E00093B1009598C19A62FF02C0949A44
:100FC00001C0C2987894D8C002E0F894B0937C0035
:100FD000E1E8F0E00093B1009398929A62FF02C0BA
:100FE000949A01C0C2987894C7C095FD0BC0F8943C
:100FF000B0937C00EBE6F0E0959862FF01C0949A14
:101000007894BAC0F894B0937C00EBE6F0E0939843
:1010100062FF01C0949A7894AFC0AC98B4E095FD9B
:101020000AC0F894B0937C00929AC19862FF01C004
:10103000949A7894A1C0F894B0937C00C19A929845
:1010400062FF01C0949A789497C0AC9AB5E082FF91
:1010500024C095FD11C001E0F894B0937C00E7E74F
:10106000F0E00093B1009498C29A62FF02C0939A94
:1010700001C09298789480C004E0F894B0937C000A
:10108000EBE8F0E00093B1009498C29A62FF02C0CE
:10109000959A01C0C19878946FC095FD0BC0F894E3
:1010A000B0937C00E5E6F0E0949862FF01C0939A6B
:1010B000789462C0F894B0937C00E1E7F0E09498F3
:1010C00062FF01C0959A789457C0AC98B6E095FD40
:1010D0000AC0F894B0937C00C19AC29862FF01C024
:1010E000939A789449C0F894B0937C00929AC298ED
:1010F00062FF01C0959A78943FC0AC9AB1E082FF3C
:1011000024C095FD11C004E0F894B0937C00EBE896
:10111000F0E00093B1009398929A62FF02C0959A12
:1011200001C0C198789428C001E0F894B0937C0085
:10113000E7E7F0E00093B1009598C19A62FF02C022
:10114000939A01C09298789417C095FD0BC0F894BB
:10115000B0937C00E1E7F0E0939862FF01C0959ABC
:1011600078940AC0F894B0937C00E5E6F0E0959896
:1011700062FF01C0939A78946F7E089524E630E070
:10118000F9012092B100939894989598929AC29AF6
:10119000C19A6B7F0895A2EBB0E009E00D9309E0DE
:1011A0000D9304E00D930FEF0D9303E00D930FEFFC
:1011B0000D930BE00D9303E00D9301E00D9301E01F
:1011C0000D93AEEBB0E001E00D930FEF0D930D9397
:1011D0000D930D930D9303E00D930FEF0D930FEF10
:1011E0000D930D9305E20D9300ED0D9308E20D9321
:1011F00000E50D9304E00D930FEF0D9302E00D93C6
:1012000000E00D930AE70D930FEF0D9300E00D93AF
:1012100001E00D9300E00D9303E00D9300E00D93CA
:1012200008952091B9008B7F233009F48460B09138
:10123000BA00B33019F09F7DB1FD90629F7BB091F1
:10124000BB00B1FD9064223011F0886001C0877F3F
:1012500008950A95E00FF21DB4910895ECE1F0E0D5
:101260000091B200F6DFB093D700ECE1F0E000911E
:10127000B300EFDFB093D800EAE2F0E00091B800ED
:10128000E8DFB093D9000091B800023008F402E022
:1012900000937300B091CE000FEFB23009F400EA72
:1012A000B33009F402E800937200E8E3F0E0009143
:1012B000D500CFDFB093A000089508952091C80015
:1012C0003091C900B091BA00B33009F43E5097FF95
:1012D00002C020E03FEFB32FB21B6B2EB25810F4C8
:1012E000B2E86B2E00E00395609EB12DBD57D8F398
:1012F0000093AC0008959068E1DFAED9ADD920E04D
:1013000030E0B0E16B2EA4D9B09196002B0F321DC6
:101310006A94C9F7B4E036952795BA95E1F7822E1D
:101320009F77CCDF0895F894E3E0F0E0B9E0B7BF31
:10133000B491B078C1F3F894A895B1B5B861B1BDD6
:10134000B0E0B1BDB4E0BEBFBFE5BDBF17DFB6E0E2
:10135000B8BBB6E1B7BBB8E0B5BBBCE1B4BBB4E069
:10136000B2BBBCE3B1BB2224A0E0B0E02D92AA3115
:10137000E9F7A0E6B0E00FEF2D920A95E9F7B1E0AA
:10138000B093A20008DF06D3B7E0B06CB7B9B6B12E
:10139000B460B068B6B90091CA000093AD00B1E086
:1013A000B0936A00F8945CD966D956D967D954D9F4
:1013B00068D952D9F8940AEF1AEFA6B396FDA09512
:1013C000A0FF1FC01A95C9F70A95B1F7E0E0FCE14C
:1013D000B591B43E39F4B591B03E21F4B591BF3F1B
:1013E00009F40CC0E0E0F395F395B591B83F49F4EA
:1013F000B591B43931F4B591BA3A19F4EE27F695AE
:1014000009940FDF2BDF59DF59DF0091CA000093E9
:10141000AD00B4DEB2E0B3BFB2E0BEBDB2E0B5BD78
:10142000B1E5B8BFB9BFB0B70B2FB77FB0BFB8B188
:10143000B0B703FDB860B0BF09D97894C8DA20927C
:101440007000BEB5B06496FDBF7BBEBDB9B7B062DB
:10145000B9BFBB27B062B8BF8D7F02D9626033E0ED
:101460002CE0B0919500BB2321F42CE03A9509F4CF
:10147000A1CFF2D880FF9ECF8E7FB0919600B23080
:1014800078F3B92FBF710091980000939700B09343
:101490009800B01729F72A9521F76D7FBEB5B06483
:1014A00096FDBF7BBEBDBB27B062B8BF8D7FB0913C
:1014B000D400BB2321F48062B92FB0709B2F8F7BA7
:1014C00020926700CBD885FF05C0B0916700BA3085
:1014D00008F08064BDD802E085FF01C000E0B09153
:1014E0009600B017B8F3F894C6D8C5D8C4D8789485
:1014F000B7D820928600B091BA00B33009F47DC00D
:10150000A7D8B091BE00B13008F477C0B0916A009E
:10151000B13008F472C085FD18C0B0919600BF3F8D
:1015200008F46BC0F894B0D8789498D8B09196002D
:10153000B130C0F7F8949FD88DD89DD878948ED8C4
:10154000B0919600BF3FB0F3E6C2B3E09B2E906827
:10155000F894B4DE789482D8F8949F77AFDE8090C8
:101560009600B0919600BF37789408F44EC06ED8BC
:10157000F8948AD878949A9451F7BDDEB82DB09338
:10158000C9006ED8F8949AD27894BAE09B2E9068ED
:10159000F89494DE789462D8F8949F778FDE8090E8
:1015A0009600B0919600BF37789478F74FD8F894AA
:1015B00062D850D860D878949A9449F79CDEB82DB8
:1015C000BB5FB093C8000B2F1091C900125810F0E8
:1015D000100B20F4B2E80B0F0093C90041D8F89427
:1015E00006D27BD278943AD8F89468DE7894B09199
:1015F0009600BF3F08F48FCF8EC200919600B09145
:1016000086000B1710F00093860028D801E0B091F7
:10161000BA00B35009F405E0B0919600B01708F095
:101620006ACFF89431D830D82FD8789419D820922E
:101630006A0020926B0020926C00B0916B00B39511
:10164000B0936B00BF3F71F5B0916C00B395B09350
:101650006C00B091CC0009E1BA9559F002E3BA955B
:1016600041F00DE7BA9529F00AEFBA9511F02092F2
:101670006C00B0916C00B017A8F080DDE7D7B09196
:101680006C00BA95B0936C0020926B00B091CB00C7
:10169000B093AD00F894F8D77894B091CA00B093A5
:1016A000AD00DCD7D7D7B0916800BB2319F485FF14
:1016B00001C080CE01E085FD01C006E0B09196003A
:1016C000B01708F4BACFB091BA00B35009F0C6D73A
:1016D000B0916800BB2309F46DCEF8944FDD2092E1
:1016E00061002092620020926300522C20926400DC
:1016F0002092A1007894B091B700BB0FB0939F00E7
:1017000020927E0020927F00209280002092810013
:10171000209282002092AA0060E070E02092710086
:10172000B8E0B093AA00706191D7B7E074FDB6E05D
:10173000B06CB7B9B6B1B068B064B6B9B6B1B6FD01
:10174000FDCF04B115B1B6B1BF77B6B9112309F019
:101750000FEF0093AB003DD9B8E0B093AA007061E1
:1017600060DDF894BFEFB0939B0092D9B091610017
:10177000B0939B00B0939C00B0939D007894B1E02F
:10178000B0936100B09363005B2EB0936400B0939C
:10179000A400B0919A00B093A300B091BA00B33006
:1017A00019F49F7D87FD90627160726020926D00D8
:1017B0008CDCA3DC86D98BD984D989D982D900DB8A
:1017C000E5D7A4DBD2DB83D9F4DA65FD18D877FF3F
:1017D000CAD877FDECD89ADBE0DB79D9F1DA65FD80
:1017E0002AD894DB1ADC73D9E4DA65FD5ED88EDB87
:1017F0002CDC6DD9E5DA65FD88D888DB66DC67D935
:10180000D8DAB7E074FDB6E0B06CB7B9B6B1B0687D
:10181000B064B6B97BDB71DC5AD9DBD871FF24C068
:10182000B0919E00B0939B00B0939C00B0919A0041
:10183000B093A300B1E0B093A40018E12CE0B09104
:101840006D00B11758F07D7F746020936F00B091E8
:101850009E00B0939B00B0939D0006C0B09196008F
:10186000B13008F0ACCF64C072FF15C066FD13C084
:10187000B0916F00BA9519F47B7F7860A0CFB093D8
:101880006F00B0919600B13008F099CFB091BA00D6
:10189000B33009F04DC020927000B09199000AEF6A
:1018A0001091D600112309F003E0B01708F040C0F2
:1018B00085FF04C0B0916800BB23D1F1B091BA009C
:1018C000B33081F495FD03C087FD04C00BC087FFD2
:1018D00001C008C066FD06C06064B0919E00B09370
:1018E0009B0082CF00EF66FF05C0B0919E00B093D1
:1018F0009B0000E2B0917B00B01708F460CF66FF58
:1019000017C06F7B9F7D87FD90627460B2E1B093DA
:101910006F00B0919E00B0939B0051CFB0917000CA
:10192000B395B0937000B0919600BB2309F002C04C
:1019300020927000F89422DC8090B900B2E0B0935D
:10194000B9006FDC8092B9002092610020926200A1
:1019500020926300522C2092640020929F0060E04D
:1019600070E078947BD60ADC0091D600002319F051
:10197000939A949A959AB7E0B06CB7B9B6B1B4603F
:10198000B068B6B985FF05C0B0917000B43008F0FA
:1019900011CD4FCEEDE0F0E023D0053509F01BC0AE
:1019A000EEE0F0E01DD00A3A09F015C03AE0A2EBF3
:1019B000B0E0E3E0F0E014D00D9331963A95D9F71A
:1019C00039E1AEEBB0E0EFE0F0E00AD00D933196F4
:1019D0003A95D9F702C0DFDB0AD0E8E2F0E00895DB
:1019E000E199FECFEEBBFFBBE09A0DB308951ED088
:1019F0003AE0A2EBB0E0E3E0F0E00D910FD03196D9
:101A00003A95D9F739E1AEEBB0E0EFE0F0E00D91B7
:101A100005D031963A95D9F712D00895E199FECFC5
:101A20000DBBEEBBFFBBE29AE19A0895EDE0F0E05A
:101A30000FEFF4DFEEE0F0E00FEFF0DF0895EDE000
:101A4000F0E005E5EBDFEEE0F0E00AEAE7DF08951D
:101A50003091AE000091AF00313011F40093B2002C
:101A6000323011F40093B300333011F40093B4001A
:101A7000343011F40093B600353011F40093B800FF
:101A8000363011F40093C400373011F40093B900DC
:101A9000383011F40093D500393011F40093CE00A2
:101AA0003A3011F40093BA003B3011F40093BB00BC
:101AB000089525E0D5D52A95E9F70895DCD5DED53A
:101AC000E0D5E2D5C7D5D7D5D9D5DBD5DDD5C2D5BB
:101AD000D2D5D4D5D6D5D8D50895D6D5D2D5CED5CC
:101AE000CAD5B8D5D1D5CDD5C9D5C5D5B3D5CCD521
:101AF000C8D5C4D5C0D508958090AE009090AF00F1
:101B0000BAD5B9D5B8D5A6D58A94D1F7BDD5A2D5C1
:101B10009A94E1F70895F894D1DF7894CADFC9DF89
:101B2000B1E0B093AE00B1E0B093AF002092B0004E
:101B3000F894E2DF7894B5E06B2E7090960090D523
:101B4000B09196007B16C9F7B13018F0BF3F40F155
:101B500007C07EDFF8944BDFB1DFB8E0B1BDA9DF8D
:101B60006A9459F7B091B000B395B093B000B33018
:101B700008F4DECF9EDFB091AF00B395B093AF0015
:101B8000F894B091AE00BA95EEE3F0E0EB0FF21DE1
:101B9000049178940395B091AF00B01708F4C6CFC4
:101BA00088DF87DFB091AE00B395B093AE00B091FF
:101BB000AE00BC3008F4B7CFEEDAF89418DFB8E026
:061BC000B1BD77DFB0CBE0
:00000001FF
